:100000000C945A040C9492040C9492040C94920450
:100010000C9492040C9492040C9492040C94920408
:100020000C9492040C9492040C94BB200C948D219B
:100030000C940F1B0C9492040C9492040C94920454
:100040000C9492040C9492040C9492040C949204D8
:100050000C9492040C94971B0C9492040C949204AC
:100060000C9492040C9492040C9492040C949204B8
:100070000C9492040C9492040C9492040C949204A8
:100080000C9492040C9492040C9492040C94920498
:100090000C9492040C9492040C9492040C94920488
:1000A0000C9492040C9492040C949204C807C80710
:1000B000F407F4075C088709870987097A08130998
:1000C00024092409FA2121221923212219236D222E
:1000D00090221923E722F6223E00165C14001A0033
:1000E0000800150017001C0018000C001200130077
:1000F0002A004B002B0004001600070009000A002C
:100100000B000D000E000F00280000004E00E10063
:100110001D001B000600190005001100100036002C
:100120003700E500000029002F61E300E2002C0009
:10013000000000002C410000E60002513071000078
:10014000010001001E001F002000210022002300EA
:100150002400250026002700010001000100010005
:1001600001000100010001005000520051004F0049
:100170000100000001000100AA00A800A900010080
:100180000100010001002D002E000100000001000F
:10019000010001000100010000000000010000005A
:1001A000010001000100000001003A003B003C009A
:1001B0003D003E003F00400041004200430044003B
:1001C00045000100010001000100010001000100E3
:1001D0000100330034003200010000000100010082
:1001E000640001000100010001000100010038006D
:1001F00001000100000001000100010001000100F8
:10020000000000000100000001000100005C00008F
:1002100044454255473A2064697361626C65642EB7
:100220000A0044454255473A20656E61626C656438
:100230002E0A000A0025303258006C65645F746134
:10024000736B3A20004F6E6573686F743A20616378
:10025000746976653A2025640A000A002530313633
:1002600062003A200025303258000A722F63203095
:100270003132333435363738394142434445460A02
:10028000003F00433E20004C25640A000A092D204F
:10029000537461747573202D0A686F73745F6B6596
:1002A00079626F6172645F6C65647328293A2025F6
:1002B0003032580A6B6579626F6172645F70726F79
:1002C000746F636F6C3A20253032580A6B6579621F
:1002D0006F6172645F69646C653A20253032580A38
:1002E00074696D65725F72656164333228293A20E2
:1002F0002530386C580A000A092D2056657273693A
:100300006F6E202D0A5649443A20307846454544C0
:1003100028456C6C696F7420506F77656C6C292070
:100320005049443A203078343634362865623436C1
:1003300029205645523A203078303030310A425523
:10034000494C443A2020284665622032372032301A
:100350003232290A4F5054494F4E533A204C554699
:10036000412045585452414B455920434F4E534F1D
:100370004C4520434F4D4D414E4420343039360AD0
:100380004743433A20352E342E30204156522D4CCF
:100390004942433A20322E302E30204156525F419E
:1003A0005243483A20617672350A000A092D2043EB
:1003B0006F6E736F6C65202D0A4553432F713A0998
:1003C000717569740A000A092D204D6167696320FF
:1003D0002D0A443A094465627567204D657373615F
:1003E000676520546F67676C650A583A094D6174F8
:1003F000726978204465627567204D6F646520548A
:100400006F67676C65202D2053686F77206B657967
:100410007072657373657320696E206D61747269A3
:100420007820677269640A4B3A094B6579626F619B
:10043000726420446562756720546F67676C65203D
:100440002D2053686F77206B657970726573732008
:100450007265706F72740A4D3A094465627567205F
:100460004D6F75736520546F67676C650A563A095E
:1004700056657273696F6E0A533A095374617475E5
:10048000730A433A09416374697661746520436F66
:100490006E736F6C65204D6F64650A46312D463171
:1004A000303A0953776974636820746F204C61791E
:1004B000657220302D392028463130203D204C30C7
:1004C000290A302D393A0953776974636820746FAB
:1004D000204C6179657220302D390A4752415645CA
:1004E0003A0953776974636820746F204C617965A9
:1004F0007220302028616C7465726E617465290AFF
:10050000423A094A756D7020746F20426F6F746CA7
:100510006F616465720A4553433A094A756D7020EC
:10052000746F20426F6F746C6F6164657220286114
:100530006C7465726E617465290A453A0950726976
:100540006E7420454550524F4D2053657474696E4A
:1005500067730A4253504143453A09436C656172DF
:1005600020454550524F4D0A006B65796D61705FB3
:10057000636F6E6669672E7261773A202530325854
:100580000A2E737761705F636F6E74726F6C5F6356
:100590006170736C6F636B3A2025750A2E6361700E
:1005A000736C6F636B5F746F5F636F6E74726F6C8D
:1005B0003A2025750A2E737761705F6C63746C5FE7
:1005C0006C6775693A2025750A2E737761705F72C2
:1005D00063746C5F726775693A2025750A2E7377AC
:1005E00061705F6C616C745F6C6775693A2025752A
:1005F0000A2E737761705F72616C745F72677569E0
:100600003A2025750A2E6E6F5F6775693A20257549
:100610000A2E737761705F67726176655F657363D9
:100620003A2025750A2E737761705F6261636B7380
:100630006C6173685F6261636B73706163653A20BC
:1006400025750A2E6E6B726F3A2025750A00646557
:100650006275675F636F6E6669672E7261773A20B5
:10066000253032580A2E656E61626C653A20257518
:100670000A2E6D61747269783A2025750A2E6B65B1
:1006800079626F6172643A2025750A2E6D6F7573F9
:10069000653A2025750A006565636F6E6669673A7D
:1006A0000A64656661756C745F6C617965723A2085
:1006B00025750A003F000A6D6F7573653A206F66F5
:1006C000660A000A6D6F7573653A206F6E0A000A3C
:1006D0006B6579626F6172643A206F66660A000A20
:1006E0006B6579626F6172643A206F6E0A000A6D01
:1006F00061747269783A206F66660A000A6D6174E7
:100700007269783A206F6E0A000A64656275673A0A
:10071000206F66660A000A64656275673A206F6E2C
:100720000A000A0A4A756D70696E6720746F20624C
:100730006F6F746C6F616465722E2E2E2000433EC5
:100740002000436C656172696E6720454550524FC9
:100750004D0A000A002530325820006B6579626F1F
:100760006172645F7265706F72743A20005B735DD2
:10077000005B575D005B535D005B525D005B445D59
:10078000005B435D000A0365006200340036000030
:10079000001C0345006C006C0069006F00740020B1
:1007A0000050006F00770065006C006C00000004D2
:1007B00003090409025B00030100A0FA0904000018
:1007C0000103010100092111010001224000070578
:1007D0008103080001090401000103000000092150
:1007E00011010001223200070582032000010904E3
:1007F0000200020300000009211101000122220071
:1008000007058303200001070503032000011201EF
:10081000000200000008EDFE464601000102000152
:100820000631FF0974A1010975150026FF00952006
:10083000750881020976150026FF0095207508913C
:1008400002C005010980A101850319012AB700151D
:100850000126B700950175108100C0050C0901A1A2
:1008600001850419012AA002150126A0029501752F
:10087000108100C005010906A101050719E029E75B
:100880001500250195087501810295017508810102
:100890000507190029FF150026FF00950675088138
:1008A0000005081901290595057501910295017545
:1008B000039101C011241FBECFEFDAE0DEBFCDBF30
:1008C00004B603FE18C08091630290916402A09167
:1008D0006502B09166028730904BA740B04B59F447
:1008E00010926302109264021092650210926602E6
:1008F000E0E0F8E3099511E0A0E0B1E0EEE5F7E40F
:1009000002C005900D92A439B107D9F722E0A4E9FD
:10091000B1E001C01D92A336B207E1F70E94D115E4
:100920000C94AD230C940000FF93EF93E09194019D
:10093000F0919501309709F00995EF91FF91089595
:10094000FC018591803011F0EFDFFBCF0895FF2788
:10095000E0E230E247FF0CC0419597FF09C0EDE2AD
:100960006095709580959095611D711D811D911DFB
:1009700027FF02C0219530E350E2AA27660F771FB8
:10098000881F991FAA1FA41710F0A41B63955A95DE
:10099000A9F7AA3008F0A95FA05DAF93F3956115A0
:1009A00071058105910541F7ED3211F4EF93F3954F
:1009B000F21718F43F93F395FBCF8F91B5DFFA95BB
:1009C000E1F70895E991F9918591803021F0853220
:1009D00019F0AADFF9CF089520E0E8945591553237
:1009E000C1F3503311F4689455915A3348F450537D
:1009F00090F3220F022E220F220F200D250FF4CF8D
:100A00000EF4219589919991533619F3533729F1B1
:100A1000533559F1BC0188279927E8945C3621F4B5
:100A20008991999168945591543639F446EF7EF046
:100A300077FF0DC08FEF9FEF0AC055374AE039F0BE
:100A4000583540E121F0523642E009F00895FF9315
:100A5000EF937DDFEF91FF91B7CFFF93EF93FC0111
:100A600081918030B9F360DFFBCFFF93EF9368DFB4
:100A7000F1CFDF93CF93CDB7DEB72596A3DFCF912C
:100A8000DF91089581E0089581E008950C94440574
:100A900008950C9448051F93CF93DF9300D000D0A6
:100AA0001F92CDB7DEB749835A836B83309197018C
:100AB00089819A81311114C0662359F0222349F0AB
:100AC0000E94C00B182F682F89819A810E94690BA0
:100AD00003C00E94940B182F69817A81812F04C072
:100AE0000E94C00B69817A810F900F900F900F9038
:100AF0000F90DF91CF911F910C94F812FC01262FDB
:100B0000408151816281738184810C944B0581E025
:100B10000895CF93DF93EC0160E00E947E05BE0153
:100B2000DF91CF910C9449050C9482140C947E149F
:100B300008950E94130A0E9498052FEF84E39CE019
:100B4000215080409040E1F700C000000C94BD1B94
:100B50000F931F93CF93DF938C0161E00E947E057A
:100B6000EC01B8010E944605882309F45BC0B80176
:100B7000CE010E94AA19882309F454C0B801CE01FD
:100B80000E94DE15882309F44DC0B801CE010E94F1
:100B90000619882309F446C0F80182818823D9F117
:100BA000CF3D8CE5D80779F140F4C115FCE5DF07AE
:100BB00091F0C130DC4591F02EC0CC35EDE5DE077B
:100BC00041F1CD35FDE5DF0709F1CB35DD4519F5FF
:100BD0000E94571020C00E94990524C080911F02D6
:100BE000C82FC095C170C0FB80F980931F02CC2331
:100BF00029F082E292E00E94A00414C080E192E019
:100C00000E94A00410C00E940B110CC00E944E1044
:100C100002C00E945A10C801DF91CF911F910F911D
:100C20000C944205C0E08C2FDF91CF911F910F9162
:100C300008950E94F11A0C9457060E945A060C94CB
:100C4000F71A8295982F937344E0949F9001112492
:100C50008C7C86958695282B822F8575880F2A7A1D
:100C60002695822B0895CF93DF93D92F0E942106DA
:100C7000C82F8D2F0E9421062C2F30E0322F2227E3
:100C8000A901482BCA01DF91CF91089508950C94D2
:100C9000460681E008950C9449060895CF93C82F25
:100CA0000E9447068C2F0E944B06CF91089580E04A
:100CB0000C944E060E94061A0C944E06CF930E9486
:100CC000061AC82F80919601C81741F1C09396016A
:100CD00080911F0282FF1EC080FF04C08AE392E061
:100CE0000E94A00480911F0280FF0CC01F92CF932E
:100CF00085E392E09F938F930E9439050F900F90A8
:100D00000F900F9080911F0280FF04C083E392E058
:100D10000E94A0048C2FCF910C944E06CF91089581
:100D2000CF93DF93CDB7DEB72B970FB6F894DEBF26
:100D30000FBECDBF4F83588769877A878B87611134
:100D40000E94860F9E012F5F3F4F86E0F9011192AE
:100D50008A95E9F785E0FE013796D90101900D9259
:100D60008A95E1F789819A814C815D81452B31F02B
:100D70009F3F31F491E08F3F19F403C091E001C02F
:100D800090E090FF09C049815A816B817C818D81FF
:100D90009E810E94A70E05C0C9010E94870581118E
:100DA000F2CF2B960FB6F894DEBF0FBECDBFDF910A
:100DB000CF910895FC01808191810E94020C0895D9
:100DC000CF93882309F44DC0C82F8CEF8C0F813A44
:100DD000F8F48C2F0E94BD18811143C06C2F8091B4
:100DE0000201909103010E94931A882349F06C2F0D
:100DF00080910201909103010E94CB1A0E94A80FDA
:100E00006C2F80910201909103010E94C91A0CC0BD
:100E100080E28C0F883058F4C77081E001C0880FE1
:100E2000CA95EAF70E94690FCF910C94A80FEBE5E1
:100E3000EC0FE33040F4F0E0E15CFE4F808190E0A5
:100E4000CF910C945B1AC85AC73158F4EC2FF0E0DC
:100E5000EE0FFF1FEF5EFE4F80819181CF910C94CA
:100E6000711ACF910895882349F1682F8CEF860F6E
:100E7000813A38F480910201909103010E94CB1ACB
:100E80000CC080E2860F883050F4677081E001C0AA
:100E9000880F6A95EAF70E946F0F0C94A80F8BE5F4
:100EA000860F833020F480E090E00C945B1A685A3F
:100EB000673120F480E090E00C94711A08951F933C
:100EC000CF93DF93182FEB010E94E006209741F0AB
:100ED0008FE99FE00197F1F700C000002197F6CF5E
:100EE000812FDF91CF911F910C943307893319F033
:100EF00060E070E002C060E570E00C945F0788235A
:100F000021F00E94690F0C94A80F0895882321F006
:100F10000E946F0F0C94A80F0895CF92DF92EF926A
:100F2000FF920F931F93CF93DF937C01D62FC72F90
:100F3000FC011281058102950F700E945F0F8823CA
:100F4000B9F01123A9F08C2F807F803421F080E24A
:100F50008D0F883068F08091410282FD09C082E0E7
:100F60000E9408100E945F0F91E0D82ED92601C080
:100F7000D12CCC2EC2948FE0C8228C2D90E08C30E6
:100F8000910508F0C4C1FC01EA5AFF4F0C945823A4
:100F90008C2F807FCF70882311F0C295C07F1123E2
:100FA00099F0CC2309F49FC180E28D0F883010F0B6
:100FB000D11104C08C2F0E94690F03C08C2F0E9496
:100FC000790F0E94A80F8FC18D2F0E943307CC2369
:100FD00009F49DC180E28D0F883038F1DD2329F1BD
:100FE0008C2F0E947F0F24C08C2F807FCF70803287
:100FF00011F0C295C07FDD2319F0D130A1F13DC0C1
:101000008091410282FF17C0112349F0CC2329F0BF
:101010008C2F0E94690F0E94A80F80E065C180E0BC
:101020000E943307CC2309F472C18C2F0E946F0FEA
:101030000E94A80F6CC1112371F0002341F0013010
:1010400031F40E94890F8C2B0E94910F60C10E9485
:10105000890F8C2B1DC0002319F0013009F457C1F2
:101060000E949E0F25C0112321F0063008F04FC1C9
:101070000EC0053008F04BC11BC0112361F00023E6
:1010800031F0F701858180FF2EC18F7085838C2F11
:101090000E947F073CC1002359F0D93309F034C1C5
:1010A000FFEF07EE13E0F15000401040E1F72AC1D6
:1010B0008C2F0E9486072BC18C2F86958695837076
:1010C00019F0813061F023C1112321F08D2F9C2F65
:1010D000937002C080E090E00E945B1A20C111234F
:1010E00021F08D2F9C2F937002C080E090E00E9431
:1010F000711A15C18C2F837009F047C011110BC1F3
:101100002D2F229526952770220F220F6D2F6F709D
:10111000862F90E0A0E0B0E0022E04C0880F991F57
:10112000AA1FBB1F0A94D2F7D4FF10C04FE050E0B3
:1011300060E070E004C0440F551F661F771F2A95BA
:10114000D2F7409550956095709503C040E050E00F
:10115000BA01C695C695C3708A019B01082B192B4D
:101160002A2B3B2BC901B801C23049F058F4C130D9
:1011700019F00E947F0ACFC00E946D0ACCC00E9465
:10118000910AC9C00E946B0AC6C0112319F08C2FA6
:10119000817001C08695882309F4BDC02D2F22954A
:1011A00026952770220F220F6D2F6F70862F90E0EB
:1011B000A0E0B0E0022E04C0880F991FAA1FBB1F39
:1011C0000A94D2F7D4FF10C04FE050E060E070E026
:1011D00004C0440F551F661F771F2A95D2F740950C
:1011E00050956095709503C040E050E0BA01C695F7
:1011F000C695C3708A019B01082B192B2A2B3B2B08
:10120000C901B801C23049F058F4C13019F00E9448
:10121000440B81C00E94320B7EC00E94560B7BC0E3
:101220000E94A50A78C0CF70112339F08C2F0E943C
:10123000CB0A8D2F0E947F076EC08D2F0E948607DC
:101240008C2F0E94EC0A67C0D23F21F128F4D03FD6
:1012500041F0D13FC1F043C0D33F19F1D43F79F001
:101260003EC0112341F0053008F051C08C2F8F7122
:101270000E94110B4CC0063008F049C0F7CF809196
:10128000410282FF18C0112339F08C2F8F710E9408
:10129000CB0A3DC01123C9F38C2F8F710E94EC0A39
:1012A00036C0112329F08C2F8F710E94B60A2FC0EF
:1012B0000E94B10A2CC0112349F0CF718C2F0E94DB
:1012C000CB0A63E08C2F0E94ED0F21C081E00E94C9
:1012D00008100230E0F082E00E94081018C01123CC
:1012E00031F0002391F28D2F0E94E00610C0002300
:1012F00099F2D93349F41FEF27EE33E01150204023
:101300003040E1F700C000008D2F0E94330788EFC6
:101310008C0D843020F40E94061A0E944E06DD20B7
:10132000C9F00E945B0F80FD15C0F70112820E9478
:10133000550F0E94CB0AC7010E94CB090E94550F8E
:10134000DF91CF911F910F91FF90EF90DF90CF90A1
:101350000C94EC0ADF91CF911F910F91FF90EF90C9
:10136000DF90CF9008950F931F93CF93DF93EC01FD
:10137000688179818A810E940D0C8C010E94680B22
:101380000E94590AB801CE010E948D07DF91CF91CA
:101390001F910F910895CF93DF93EC01988189817C
:1013A0002B813C81232B31F08F3F31F481E09F3F33
:1013B00019F403C081E001C080E080FD1DC0CE01B2
:1013C0000E94A805811110C00E945F0F8823A1F020
:1013D0008A81882389F08091410282FD0DC082E0DC
:1013E000DF91CF910C940810CE010E94B309CE0179
:1013F000DF91CF910C948905DF91CF91089580E022
:1014000090E00E945B1A80E090E00E94711A0E94B6
:10141000860F0C94A80F80910201909103010E9405
:10142000CD1A0C94FF090E94760F0C940B0A92952A
:101430009F70963079F010F4925001C09A5092301B
:1014400068F4803F69F018F4883E40F409C0843F96
:1014500029F406C0883E20F0813F11F080E0089515
:1014600081E00895FC01808191810E94020C0E941C
:10147000170A0895CF93DF9300D000D01F92CDB705
:10148000DEB70F900F900F900F900F90DF91CF91DC
:101490000895CF93DF9300D000D000D0CDB7DEB752
:1014A00026960FB6F894DEBF0FBECDBFDF91CF9169
:1014B0000895089508950C945A0A0C945B0A0E94AA
:1014C0005D0A6093BF017093C0018093C101909346
:1014D000C2010C94FF090C945F0A0F931F930091B3
:1014E000BF011091C0012091C1013091C201602B58
:1014F000712B822B932B1F910F910C945F0A0F93EA
:101500001F930091BF011091C0012091C101309142
:10151000C20160237123822393231F910F910C94A6
:101520005F0A0F931F930091BF011091C00120919A
:10153000C1013091C20160277127822793271F9133
:101540000F910C945F0A0C945A0A0E94A30A6093AC
:10155000BB017093BC018093BD019093BE010C94BC
:10156000FF0960E070E0CB010C94A50A0F931F9374
:1015700041E050E060E070E08A019B0104C0000F90
:10158000111F221F331F8A95D2F7C901B8011F917D
:101590000F910C94A50A0F931F9341E050E060E077
:1015A00070E004C0440F551F661F771F8A95D2F75D
:1015B0008091BB019091BC01A091BD01B091BE0191
:1015C0008A019B01082B192B2A2B3B2BC901B8013F
:1015D0001F910F910C94A50A0F931F9341E050E0C7
:1015E00060E070E004C0440F551F661F771F8A95A6
:1015F000D2F740955095609570958091BB01909180
:10160000BC01A091BD01B091BE018A019B010823DC
:1016100019232A233B23C901B8011F910F910C9470
:10162000A50A0F931F9341E050E060E070E004C012
:10163000440F551F661F771F8A95D2F78091BB0113
:101640009091BC01A091BD01B091BE018A019B01A6
:10165000082719272A273B27C901B8011F910F9195
:101660000C94A50A0F931F930091BB011091BC012C
:101670002091BD013091BE01602B712B822B932BE9
:101680001F910F910C94A50A0F931F930091BB011A
:101690001091BC012091BD013091BE0160237123E6
:1016A000822393231F910F910C94A50A0F931F93EC
:1016B0000091BB011091BC012091BD013091BE0190
:1016C00060277127822793271F910F910C94A50AF9
:1016D00008952DE0929F800D1124E82FE695E69560
:1016E000E695877051E001C0550F8A95EAF785E0CD
:1016F000E89FF0011124E856FE4F20E030E070E052
:101700004081CB01022E02C0969587950A94E2F79C
:101710008170819584278523842781932F5F3F4F94
:101720002530310569F708952DE0929F800D112431
:10173000682F669566956695982F977085E0689FE7
:10174000B001112440E050E080E0FB01E40FF51F00
:10175000E856FE4F208130E0092E02C036952795CD
:101760000A94E2F721703327042E01C0220F0A9455
:10177000EAF7822B4F5F5F4F4530510531F70895EF
:10178000BF92CF92DF92EF92FF920F931F93CF936E
:10179000DF938C01C090BB01D090BC01E090BD01F3
:1017A000F090BE018091BF019091C001A091C10154
:1017B000B091C201C82AD92AEA2AFB2ACFE1D0E097
:1017C000D701C6010C2E04C0B695A79597958795AD
:1017D0000A94D2F780FD04C0219790F7B12C07C07E
:1017E000BC2EB8018C2F0E940B130197A9F38B2DEF
:1017F000DF91CF911F910F91FF90EF90DF90CF90ED
:10180000BF900895CF93DF93EC010E94C00BBE01FF
:101810000E940B13DF91CF9108951F93CF93DF9315
:10182000EB0190919701992321F0CB010E94020CCA
:1018300013C0882349F0CB010E94C00B182F682FDA
:10184000CE010E94690B04C0CB010E94940B182F9B
:10185000BE01812F0E940B13DF91CF911F9108953C
:101860001F93CF93DF93C091C30116E08091C40111
:10187000C81799F0D0E01C9FF0011D9FF00D1124B6
:10188000EB53FE4F40815181628173818481958148
:101890000E94490A2196C770E9CFDF91CF911F912D
:1018A00008954091F5015091F6016091F701709112
:1018B000F8018091F9019091FA010C94490AEF9294
:1018C000FF920F931F93CF93DF938091FA0182953C
:1018D0008F7009F065C08091F701882309F460C01A
:1018E0008091C301F090C4011091F5010091F601BF
:1018F0006091F8017091F90191E01F3F09F090E0CB
:10190000C0910001D0910101292F96E0E92E8F1599
:1019100009F446C06115710521F00F3F21F030E058
:1019200003C031E001C0322F90E030FD36C0E89EA8
:10193000F001E99EF00D1124DF01AB53BE4F11966B
:101940003C911197301329C03C91311326C0129657
:101950003C911297311121C013964D915C911497CF
:10196000461B570B4C175D07C0F48091FA018F702E
:1019700080618093FA01E653FE4F80818F70806111
:10198000808385EF91E00E94CB09DF91CF911F9179
:101990000F91FF90EF900C94300C01968770B7CFA9
:1019A000DF91CF911F910F91FF90EF9008959F923B
:1019B000AF92BF92CF92DF92EF92FF920F931F935D
:1019C000CF93DF93CDB7DEB761970FB6F894DEBF44
:1019D0000FBECDBF8C0185E0F801DE011D960190A0
:1019E0000D928A95E1F7D8011296EC909091F5014D
:1019F000E091F6012091F8013091F90121153105AE
:101A000031F0EF3F31F481E09F3F19F403C081E0F2
:101A100001C080E0B82FB1709B2E80FD47C1D80176
:101A20004C9111965C9111971396AD90BC901497C0
:101A300085EFC82E81E0D82EF090F701B501621B2A
:101A4000730B2091000130910101FF2009F4D9C0EE
:101A50008091FA016217730708F095C0282F207F44
:101A600009F052C05E1313C0491311C0FE2CE110DF
:101A70000EC08F7080618093FA010E94510CC601E4
:101A80000E94CB098091FA01F80185834DC1AB28F2
:101A900031F05F3F31F481E04F3F19F403C081E042
:101AA00001C080E080FD03C081E08E2502C080E09F
:101AB00090E0F82FF170FF2E80FF1CC08091C301D1
:101AC0002091C40136E0821709F40BC190E0389FE1
:101AD000F001399FF00D1124EB53FE4F6181561335
:101AE00006C06081461303C06281E61203C00196FE
:101AF0008770E9CFFE2CEE2009F416C18091FA011F
:101B000081608093FA0154C05E1306C0491304C07B
:101B1000E11002C0F80199C0C8010E94320A88236E
:101B200061F1EE2051F12091FA01822F82958F70A0
:101B300090E0029774F08091F5019091F6019887FA
:101B40008F831986BB86AA862C87CE0107960E94B2
:101B5000CB0986E0F801A5EFB1E001900D928A95DE
:101B6000E1F70E945F0C0E94510C0AC05E1711F150
:101B7000C8010E94320A81112CC0C8010E94CB0901
:101B8000FF24F394D1C0282F207F81F77A2DB98AC2
:101B9000A88A6E2D89890E943A0A85EF91E00E94F9
:101BA000CB0986E0D6011D928A95E9F70E94510C77
:101BB000F12CBAC04913DCCFE110DACFF8018583EC
:101BC000C8010E94CB0986E0D6011D928A95E9F7EB
:101BD000ABC0EE2091F22091FA01822F82958F7096
:101BE00090E002970CF4B5CF8091F5019091F60149
:101BF0009A8389831B82BD82AC822E83CE0101969B
:101C0000A6CF6217730708F044C0FE2CEE2009F43B
:101C1000B4CF5E1330C049132EC02091FA0120FDCD
:101C200021C0822F82958F70482F50E041155105B9
:101C3000C9F0F80125834F30510541F08F5F982F8F
:101C40009295907F822F8F70892B8583C8010E9487
:101C5000CB0986E0F801A5EFB1E001900D928A95DD
:101C6000E1F73CC086E0F801A5EFB1E001900D92EC
:101C70008A95E1F759C0C8010E94320A811169CFE3
:101C80008091FA0181608093FA01C8010E94CB091A
:101C90004BC07A2DB98AA88A6E2D89890E943A0A8A
:101CA00086E0D6011D928A95E9F718C0EE2009F466
:101CB00064CFC8010E94320AF82E882309F45DCF50
:101CC00086E0F801A5EFB1E001900D928A95E1F769
:101CD00085EF91E00E94DA060E945F0C0E94510C91
:101CE00023C04D875E878D859E850E94020C292F1B
:101CF00022952F70223028F49F7039F0811105C091
:101D00000BC0243028F49F7049F4805E883020F0A6
:101D1000C8010E94CB099F2CF92C06C0D80115964A
:101D20009C91907F91F7F8CF8F2D61960FB6F89424
:101D3000DEBF0FBECDBFDF91CF911F910F91FF90FE
:101D4000EF90DF90CF90BF90AF909F9008951F933A
:101D5000CF93DF93CDB7DEB72C970FB6F894DEBFE5
:101D60000FBECDBF4F83588769877A878B879C8743
:101D7000CE0107960E94D70C8823D1F09F818885D9
:101D80002A853B85232B31F08F3F31F481E09F3F43
:101D900019F403C081E001C080E080FD47C04F819D
:101DA000588569857A858B859C850E94490A3EC045
:101DB00086E0FE013796DE01119601900D928A951C
:101DC000E1F7FF81E8856A857B856115710531F052
:101DD000EF3F31F481E0FF3F19F403C081E001C01F
:101DE00080E080FD23C02091C40130E0C90101964C
:101DF000877099274091C30150E084179507F1F14E
:101E0000F983EA837D836C8396E0929FD001939F50
:101E1000B00D1124AB53BE4FFE01319601900D92CF
:101E20009A95E1F78093C4010E94300C16E08091EE
:101E3000C3019091C401891771F1189FC001112449
:101E40008B539E4F0E94D70C882329F1E091C30148
:101E50001E9FF0011124EB53FE4F4081518162819E
:101E60007381848195810E94490A8091C30190E029
:101E70000196877099278093C301D9CF0E94130AD6
:101E80001092C4011092C301E5EFF1E086E0DF019A
:101E90001D928A95E9F72C960FB6F894DEBF0FBE17
:101EA000CDBFDF91CF911F91089580910302859559
:101EB0008595859508958091030287700895909186
:101EC0000302977081E009F480E0089580910E028A
:101ED000089590910E02892B80930E0208958095AB
:101EE00090910E02892380930E02089510920E02A3
:101EF000089590910D02892B80930D02089580958D
:101F000090910D02892380930D02089510920D0285
:101F1000089580910402089508950C948C0F0C94F8
:101F20008D0F9091410292FD08C090910402981784
:101F300021F0809304020C948F0F08958091040285
:101F4000882329F01092040280E00C948F0F0895EA
:101F5000CF93DF93E0910201F091030180910E0293
:101F60008083E0910201F0910301908180910D0244
:101F7000892B808380910402882381F0E091020103
:101F8000F09103019081892B8083809102019091CF
:101F900003010E94871A81110E949E0FC0910201C5
:101FA000D091030148E050E06BEF71E0CE010E9458
:101FB0005E23892B69F088E0FE01ABEFB1E0019070
:101FC0000D928A95E1F7CE01DF91CF910C94121A10
:101FD000DF91CF9108950C948C0F9091410292FD66
:101FE00010C098E0899F90011124262B20930302B2
:101FF0000E94CB0A809103028595859585950C9466
:10200000EB0F0C94CB0A1092030280E00C94EB0FC0
:10201000209103028095822380930302982F97706A
:1020200099F430E0482F082E000C550B2417350783
:1020300059F09091410292FD07C08595859585954F
:102040000E94EC0A0C9403100895CF9390914102E2
:1020500092FB222720F92817F9F0C82F892FC0FBFF
:1020600082F98093410280914002909141020E9446
:10207000871082E00E94081080911F0280FF0CC030
:102080001F92CF9385E492E09F938F930E9439052E
:102090000F900F900F900F90CF9108958091410273
:1020A00082FB882780F991E089270C94251081E034
:1020B0000C94251080E00C9425106FEF7FEF80E0EA
:1020C00090E00C94972380E090E00E94732321E03D
:1020D000893E9E4F09F020E0822F089582E090E033
:1020E0000C946B2383E090E00C946B23CF9384E0FB
:1020F00090E00E946B23C82F82E290E00E946B2345
:102100002C2F30E0A901582BCA01CF910895CF930D
:10211000C92F682F84E090E00E9479236C2F82E21F
:1021200090E0CF910C947923AB01BC018FE090E05B
:102130000C948B23AB01BC0183E190E00C948B23C6
:1021400060E070E0CB010C949A1060E070E0CB018D
:102150000E9494100C94A01069EE7EEF80E090E055
:102160000E94972360E082E090E00E94792360E083
:1021700083E090E00E9479231092BF011092C00189
:102180001092C1011092C20160E084E090E00E94D0
:10219000792360E082E290E00E94792360E085E0AC
:1021A00090E00E94792360E086E090E00E9479232D
:1021B0006FEF87E090E00E94792340E050E0BA01A1
:1021C00088E090E00E948B2360E08DE090E00E9428
:1021D000792340E050E0BA0188E190E00E948B232F
:1021E00060E087E190E00E94792340E050E0BA018E
:1021F0008CE190E00E948B2360E070E080E290E050
:102200000E94972340E050E0BA0188E190E00E94EC
:102210008B230C94A5100C94AC10682F8EE090E0EA
:102220000C9479230E947C1B60931B0270931C0208
:1022300080931D0290931E02609317027093180200
:102240008093190290931A02089585B7806885BF1C
:1022500085B7806885BF089581E008950C942C119E
:1022600008950C9430110C9430110C9433110C948B
:1022700030110C9437110C9430110E94251186E90D
:102280009DE10E94FC190E943B110C9439110E949F
:1022900031110C9430110E94FF130C944D060E94D2
:1022A000671B0E942A150E944B110C9435115F92F6
:1022B0006F927F928F929F92AF92BF92CF92DF9256
:1022C000EF92FF920F931F93CF93DF93CDB7DEB7BB
:1022D0002A970FB6F894DEBF0FBECDBF0E943F1500
:1022E000C82E81110E9412113FE0832E32E0932EFE
:1022F00000E010E0502E802F0E9423145C01F401B6
:10230000619071904F016826792661147104B1F4CF
:102310000F5F1F4F0430110569F78FEF89838A83A0
:102320001B820E94701B8160782F9D838C83498162
:102330005A816B818D810E9490063AC080911F0264
:1023400081FD0E942C14D12CEE24E394F12CC301C6
:102350008E219F21892B29F10E942E118823A9F01B
:10236000DE825F82AE20BF2081E0AB2809F480E0EE
:1023700088870E94701B8160782F9A8789874E8199
:102380005F8168858A850E949006000F111FF80101
:10239000E15FFD4F80819181E826F926F182E0829C
:1023A00007C0D394EE0CFF1CFDE0DF12D0CFB0CFFE
:1023B00081E0C11001C080E02A960FB6F894DEBF1C
:1023C0000FBECDBFDF91CF911F910F91FF90EF9086
:1023D000DF90CF90BF90AF909F908F907F906F9045
:1023E0005F9008950E9457110C945E06CF93DF937F
:1023F0000E941013EC01811522E59207E8F5811582
:1024000031E5930708F0B6C0883E910528F5803E77
:10241000910508F0E9C0883A910570F4853A910574
:1024200008F07AC08130910509F473C008F4D9C06E
:10243000049708F0D9C0D5C08F3B910508F0D1C0F2
:10244000C85AD0E0CC0FDD1FCE5BDE4F0990D8819B
:10245000C02DCE019464C9C0811540E5940708F0F1
:1024600069C0811550E4950708F060C09A95811500
:102470009F4108F4B9C0B5C0811536E5930728F52A
:10248000811545E5940708F092C0811554E595073C
:1024900008F087C0AC0143705527282F2695269554
:1024A000C115D34508F06CC081E090E002C0880FF0
:1024B000991F4A95E2F740E2249F90011124EC0114
:1024C000C22BD32BCE019C6890C081152AE59207C0
:1024D00080F4811539E5930708F072C0811548E54D
:1024E000940708F47EC0D82FCC27CE01806F906A65
:1024F0007CC090568115904208F073C08D2F8F716B
:102500000E94A413DD27D0628F71AE01582BCA013F
:102510006CC081E090E069C0C55AD0E0C059DE4F80
:102520008881C82FD0E0CE0190645FC0DF70CE01FB
:10253000906A5BC074E0969587957A95E1F7282FAD
:1025400023703C2F337081E090E002C0880F991F08
:102550003A95E2F79C68AC01522B9A019C2F9F7030
:102560009695969550E2959FE0011124C9018C2B18
:102570009D2B3BC0D82FCC27CE01816F906A35C0F0
:1025800081E090E002C0880F991F4A95E2F750E27F
:10259000259F90011124EC01C22BD32BCE019A6808
:1025A00024C0D82FCC27CE01846F906A1EC00E9411
:1025B000A4138F7190E0D82FCC27CE01906215C064
:1025C0008F700E94A41394E0D695C7959A95E1F771
:1025D000CF70D0E0DC2FCC27D0699E01282BC90119
:1025E00004C080E090E001C0CE01DF91CF9108955A
:1025F00024E3829FC0011124FC012DE0729FE00DB5
:10260000F11D1124E60FF11DEE0FFF1FE852FF4FE1
:102610008591949108950E94F8120E94F6110895F0
:102620008238910569F1B0F48133910509F46DC0E8
:1026300048F48932910509F463C08A32910509F49E
:1026400069C008958533910509F455C08933910512
:10265000B9F00895833E910569F138F4803E910503
:10266000B1F0823E910509F10895863E9105A9F1E8
:10267000873E9105B9F1843E910509F064C023C0FD
:102680002091400220FD4FC021FD4DC00895809152
:10269000400280FD44C08091410280FF44C080918F
:1026A000400284FD42C083EE4DC08091400282FF13
:1026B00038C0F5CF8091400282FD33C08091410245
:1026C00080FD31C0ECCF8091410281FF32C080910A
:1026D000400284FD2AC087EE35C08091400283FF0E
:1026E00026C0F5CF8091400283FD21C08091410238
:1026F00081FD1FC0ECCF8091400285FD1CC01DC034
:102700008091400285FD19C016C08091400286FD6F
:1027100016C017C08091400286FD13C010C089E327
:1027200011C082EE0FC080EE0DC080E00BC086EEBF
:1027300009C084EE07C089E205C085E303C08AE2D0
:1027400001C081E390E008959091400292FF0DC096
:10275000282F2871283019F4877F846006C0282F1D
:102760002471243011F48B7F886093FF0DC0282FD3
:102770002871283119F4877E846106C0282F2471BE
:10278000243111F48B7E88612091410220FF0DC01D
:10279000382F3871383019F4877F816006C0382FA0
:1027A0003171313011F48E7F886021FF0DC0282FE8
:1027B0002871283119F4877E816106C0282F217184
:1027C000213111F48E7E886194FD877E08950C94EA
:1027D0005D100E943F158FE39CE90197F1F700C05F
:1027E00000000E943F1580E00E94231480FF04C077
:1027F0000E94E7130C94BD1B08950C94E9130E94EA
:102800006310811102C00E940B110E946E10809310
:102810001F020E94761090934102809340020E9412
:10282000FD130E947210682F70E080E090E00E941B
:102830006B0A6091BB017091BC018091BD019091C8
:10284000BE010C94A30AE82FF0E0EE0FFF1FE65B39
:10285000FD4F808191810895CF92DF92EF92FF9298
:102860000F931F93CF93DF938AE692E00E94A00418
:102870008AE4E82E82E0F82EC0E0D0E095E6C92E8A
:1028800092E0D92E0CE512E0DF93CF93DF92CF9246
:102890000E94390582E692E00E94A004F70181912E
:1028A00091917F010E9433069F938F931F930F9303
:1028B0000E9439058AE592E00E94A00421968DB716
:1028C0009EB708960FB6F8949EBF0FBE8DBFC4305A
:1028D000D105D1F6DF91CF911F910F91FF90EF902D
:1028E000DF90CF90089580EA8A95F1F7089500C0AF
:1028F00008950C94731408950C947B140C947C1418
:102900000C947B140C948014F894E82FE295EF70EB
:10291000F0E031A1282F2F7081E090E001C0880FF6
:102920002A95EAF7982F9095932391A392A1892B4A
:1029300082A3789408950F931F93CF93DF93C0E8F9
:10294000D1E089918F3F11F00E94841481E0C43856
:10295000D807B9F7C3E7D1E000E811E089918F3FCC
:1029600011F00E9484140C171D07C1F7DF91CF915D
:102970001F910F910895BF92CF92DF92EF92FF9235
:102980000F931F93CF93DF938C01C62FD0E0CE011E
:1029900080589E4F6C01FC0190819F3F09F450C00C
:1029A000B62EF894E92FE295EF70F0E081A19F70C8
:1029B00021E030E001C0220F9A95EAF7822B81A333
:1029C00082A12095282322A378940E947714E3E71C
:1029D000F1E040E851E021E030E0E12CF12C6191A0
:1029E0006F3F89F0A62FA295AF70B0E090968C91C2
:1029F00090E06F7002C0959587956A95E2F780FD2B
:102A000002C0C90102C080E090E0E82AF92A220F42
:102A1000331F4E175F0719F7F60180818F3F11F0C2
:102A20000E94841461E0E114F10409F460E08B2D4C
:102A30000E947914CC0FDD1FC00FD11FF982E882EC
:102A4000DF91CF911F910F91FF90EF90DF90CF908A
:102A5000BF9008950E949B1488E0EAE4F2E0DF0151
:102A6000982F1D929A95E9F7E2E4F2E0DF011D92BA
:102A70008A95E9F784E00E948A150C949405FF92E8
:102A80000F931F93CF93DF93CDB7DEB728970FB681
:102A9000F894DEBF0FBECDBF8E010F5F1F4F88E0E1
:102AA000F80111928A95E9F7F12C6F2DC8010E9467
:102AB000BB14F394F4E0FF12F8CF48E050E0B80103
:102AC00082E492E00E945E23FF24F394009709F4CD
:102AD000F12C892B41F088E0F801A2E4B2E00190EA
:102AE0000D928A95E1F72F2D44E06AE472E082E4CA
:102AF00092E00E948B150E9496058F2D28960FB6A6
:102B0000F894DEBF0FBECDBFDF91CF911F910F9123
:102B1000FF9008950895FF920F931F93CF93DF9333
:102B2000F82E092F162FD72FC42F222349F081E02A
:102B3000809322020E94701B9093210280932002B6
:102B4000809122028823D9F0809120029091210265
:102B50000E94881B059798F0EF2DF02FA12FBD2F15
:102B600080E090E04C2F50E08417950734F42191D9
:102B700031912D933D930196F7CF10922202DF9170
:102B8000CF911F910F91FF9008950E94121E0E94F5
:102B90004F110C941E1E0E94221E0E94F2110C94D2
:102BA000401E0E940E1B0E94F91D0E943D110E94B2
:102BB000C5150E94CB150E944711FBCFCF93DF9321
:102BC000EC01FB018281882309F43CC1C430FDE59E
:102BD000DF0760F4CB3F9CE5D90788F49E012250C3
:102BE0003C452431310508F02EC109C0C236EDE55F
:102BF000DE0729F0C63AFDE5DF0709F024C10E948F
:102C000076109093410280934002C1318CE5D80741
:102C100009F4C6C008F042C0C930ECE5DE0709F48B
:102C20009BC000F5C5308CE5D80709F485C078F461
:102C3000C330ECE5DE0709F478C008F07AC0C23092
:102C4000DC4509F0F5C0809140028160EFC0C730DB
:102C50009CE5D90709F478C008F07AC08091400259
:102C60008061E4C0CD30FCE5DF0709F487C058F48B
:102C7000CB309CE5D90709F479C008F07BC080917E
:102C8000400288606FC0CF30FCE5DF0709F480C0E8
:102C900008F082C080914002877FC8C0CE3F9CE58B
:102CA000D90709F471C000F5C531FCE5DF0709F467
:102CB00085C068F4C3319CE5D90709F475C008F0F4
:102CC00095C00E94130A809140028F77AFC0CC3F1D
:102CD000FCE5DF07A9F108F054C0CB3FDC4509F063
:102CE000A7C08091410240C0C230EDE5DE0709F483
:102CF00089C058F4C1158DE5D80709F45AC008F009
:102D000069C08091410282602FC0C236EDE5DE07C6
:102D100009F47CC0C63AFDE5DF0709F481C0C33081
:102D2000DD4509F085C080E06EC080914002826080
:102D30007DC08091400216C080914002886076C0BC
:102D40008091410282604FC08091400280626EC0DB
:102D50008091400280646AC00E94130A8091400200
:102D6000806864C0846062C081603DC08091400220
:102D70008E7F5CC0809140028D7F58C08091400260
:102D800016C08091410218C0809141028D7F2BC0F6
:102D9000809140028F7E4AC0809140028F7D46C064
:102DA000809140028F7B42C080914002877F8B7F61
:102DB0003DC0809141028D7F8E7F15C08091400281
:102DC00082FB222720F991E0922790FB82F990FB69
:102DD00083F92CC080914102982F909591708E7F3D
:102DE000892B90FB81F98093410222C00E94130A33
:102DF0008091400287FB222720F991E0922790FBE7
:102E000087F914C081E00E940D1112C08091400228
:102E100084FB222720F991E0922790FB84F906C0D9
:102E200080914002982F909590FB80F9809340020A
:102E300080914002909141020E9487100E94130AE3
:102E400080E001C081E0DF91CF910895CF93C82F3A
:102E50001F928F9387E892E09F938F930E9439058A
:102E600081E090E0A0E0B0E0BC01CD0104C0660FBD
:102E7000771F881F991FCA95D2F70E946B0A0F907F
:102E80000F900F900F90CF910C94130AEF92FF9236
:102E90000F931F93CF93DF938B3109F4EDC008F0AC
:102EA0008EC08B3009F4B1C008F078C0863009F4C8
:102EB000AFC020F4853009F4BDC04EC1873009F49D
:102EC000C0C0883009F048C10E9472101F928F93D1
:102ED00087E996E09F938F930E9439050E946E10B8
:102EE00083FB992790F91F929F9382FB992790F972
:102EF0001F929F9381FB992790F91F929F93982F80
:102F000091701F929F931F928F938EE496E09F93F0
:102F10008F930E9439050E94761087FB222720F9A3
:102F20001F922F9386FB222720F91F922F9385FB58
:102F3000222720F91F922F9384FB222720F91F922A
:102F40002F9383FB222720F91F922F9382FB2227A6
:102F500020F91F922F9391FB222720F91F922F9384
:102F6000292F21701F922F9381FB222720F91F9276
:102F70002F93282F21701F922F939F938F9389E671
:102F800095E09F938F930E9439058DB79EB78896E1
:102F90000FB6F8949EBF0FBE8DBF35C0803109F4C7
:102FA00095C020F48E3009F47BC0D6C0863109F478
:102FB000A8C0893109F0D0C087EF92E084C08A327E
:102FC000E1F060F4873209F4C3C028F48E3108F4CC
:102FD000C3C08D51BEC0893269F1BEC0833448F48C
:102FE0008A3308F0B3C0853309F4B2C0883369F07E
:102FF000B3C0833409F4ACC0AFC082E497E00E9450
:10300000A0040E940B11C1E0ACC086EC93E05BC051
:1030100080911F02817F8E7F80931F028BEA93E055
:103020000E94A0048EE397E00E94A00481E08093B8
:103030002302E9CF82E297E00E94A0040E94990552
:10304000E2CF80911F02C82FC095C170C0FB80F9EC
:1030500080931F02CC2329F086E197E00E94A00410
:1030600080C089E097E00E94A00480911F02897FC0
:10307000877F80931F02C7CF90911F0291FBCC27BF
:10308000C0F981E0C827892FC0FB81F980931F0216
:10309000CC2319F08CEF96E029C08EEE96E013C099
:1030A00090911F0292FBCC27C0F981E0C827892F9D
:1030B000C0FB82F980931F02CC2319F08FED96E0BC
:1030C00015C08FEC96E00E94A0049DCF90911F0246
:1030D00093FBCC27C0F981E0C827892FC0FB83F977
:1030E00080931F02CC2351F083EC96E00E94A00451
:1030F00080911F02816080931F0233C086EB96E0AF
:10310000E2CF0E947C1B162F072FF82EE92ED091BC
:103110003F02C09110010E94061AEF92FF920F9396
:103120001F931F92DF931F92CF931F928F938CE870
:1031300092E09F938F930E9439058DB79EB70C96AE
:103140000FB6F8949EBF0FBE8DBF5DCF895301C0EF
:1031500080E00E94261757CF84EB96E00E94A004DF
:10316000C0E08C2FDF91CF911F910F91FF90EF90D6
:10317000089580E008950C94B918CF93C82F8091DA
:103180002302882319F0813031F038C00E94660F85
:103190008232B1F504C00E94660F823261F48C2F36
:1031A0000E94BB18811104C08C2F0E94461724C0B6
:1031B00081E090E021C08C2F0E94B91881111BC0C2
:1031C000C43189F018F4CB3029F010C0C93259F05D
:1031D000C83361F48BEA93E00E94A00483E892E094
:1031E0000E94A00408C0109223020CC081E892E063
:1031F0000E94A00407C081E0817006C010922302E3
:1032000080E002C080E0F8CFCF910895CF93DF93A4
:1032100086319C4541F5EB010E94660F982F8A810B
:103220002091020130910301882379F09A7A81E09C
:1032300009F480E080932402911102C069E201C088
:1032400065E3C9010E94C91A0AC080912402811154
:1032500002C069E201C065E3C9010E94CB1A0E9465
:10326000A80F80E001C081E0DF91CF9108950F9316
:103270001F93CF93DF93C42FD22FFC018281882329
:10328000C9F0409327020E94701B909326028093FE
:10329000250280E28C0F883008F057C0C77081E0AB
:1032A00001C0880FCA95EAF7DF91CF911F910F9166
:1032B0000C947F0780912702481330C0809125022B
:1032C000909126020E94881B883C910538F510E2F7
:1032D0001D0FCD17B9F080E28C0F883040F4C77015
:1032E00081E001C0880FCA95EAF70E94860718306E
:1032F00028F581E09D2F977001C0880F9A95EAF715
:103300000E947F07802F0E9476071830F0F4D77054
:1033100081E001C0880FDA95EAF70AC080E28C0FDD
:10332000883098F4C77081E001C0880FCA95EAF729
:10333000DF91CF911F910F910C948607802FDF9121
:10334000CF911F910F910C947607DF91CF911F9130
:103350000F9108950F939C01CB01243F4CE5340756
:1033600031F188F4293DFCE53F07D9F02A3D4CE5D1
:10337000340779F1283D3C45A9F506E221EE41EEFE
:1033800068ED7CE52BC0263FFCE53F07E1F0A8F0A7
:10339000273F3C4539F507E225EE46EE67EF7CE531
:1033A0001DC007E225EE45EE69ED7CE517C006E29B
:1033B00021EE40EE64EF7CE511C007E225EE44EE1D
:1033C00065EF7CE50BC006E221EE42EE66EF7CE5A0
:1033D00005C008E221E045EE6AED7CE50E94371960
:1033E00080E008C0FC018281882319F01092270236
:1033F00001C081E00F91089590939501809394010D
:10340000089590932D0280932C020895E0912C0250
:10341000F0912D02309721F00190F081E02D099478
:1034200080E00895EF92FF920F931F93CF93DF9365
:10343000E0912C02F0912D023097B1F18C010280C5
:10344000F381E02D099580911F0282FF2DC080FF3E
:1034500004C08BE597E00E94A004E80118E085E530
:10346000E82E87E0F82E80911F0280FF0BC0888134
:103470001F928F93FF92EF920E9439050F900F9049
:103480000F900F90115021961111EDCF80911F02D6
:1034900080FF0AC083E597E0DF91CF911F910F91E4
:1034A000FF90EF900C94A004DF91CF911F910F91AA
:1034B000FF90EF90089520912A0230912B02281757
:1034C000390771F090932B0280932A02E0912C022D
:1034D000F0912D02309721F00680F781E02D0994BC
:1034E000089520912802309129022817390771F098
:1034F0009093290280932802E0912C02F0912D02F2
:10350000309721F00084F185E02D09940895FC01A5
:10351000329697E080E0915029F021912223D9F34F
:103520008F5FF9CF0895662349F0FC013296089623
:103530002191621729F0E817F907D1F780E0089583
:1035400081E008959C01FC0132969FEF80E041915B
:10355000461789F09F3F19F4411101C0982F8F5FE2
:103560008630A9F79F3F39F0F901E90FF11D97FD6A
:10357000FA956283089508959C012A5F3F4FFC01EC
:103580004281461301C01282019682179307B9F750
:1035900008950C94A21A0C94BC1A029626E0FC0121
:1035A00011922A95E9F7089508950C94D41A83E0AE
:1035B00080932E020C94D51A811102C081E001C0C3
:1035C00082E080932E020C94D51A0C94DC1A81E0D0
:1035D00080932E020C94D51A0C94E71A08950C943B
:1035E000EE1A0C94EF1A0C94EE1A0C94EE1A0C943A
:1035F000EE1ACF930E94F51A0E943F150E94F31A0B
:10360000C0E08C2F0E942314892B29F4CF5FC43093
:10361000C1F780E001C081E0CF91089508951F9225
:103620000F920FB60F9211248F939F93AF93BF9376
:1036300080912F02811113C0809152029091530208
:10364000A0915402B09155024196A11DB11D8093E5
:10365000520290935302A0935402B0935502BF912B
:10366000AF919F918F910F900FBE0F901F90189563
:1036700080915A02843031F10E94190610922F0273
:1036800020E488E190E00FB6F894A895809360005C
:103690000FBE2093600083B7817F846083BF83B7B0
:1036A000816083BF7894889583B78E7F83BF0FB680
:1036B000F894A895809160008861809360001092D2
:1036C00060000FBE08950E94130A0C941D0682E04C
:1036D00084BD93E095BD9AEF97BD80936E000895E9
:1036E0002FB7F8948091520290915302A091540206
:1036F000B09155022FBF08952FB7F89460915202F0
:103700007091530280915402909155022FBF0895F9
:103710009C014FB7F8948091520290915302A0916E
:103720005402B09155024FBF821B930B08957894B9
:103730001F920F920FB60F9211248F939F93AF9306
:10374000BF938091520290915302A0915402B09184
:1037500055020196A11DB11D809352029093530210
:10376000A0935402B0935502BF91AF919F918F9156
:103770000F900FBE0F901F90189581E08093E0008E
:1037800080E28093D8001092C9008FE19EE40197F7
:10379000F1F700C0000087E090EBDC01809363024A
:1037A00090936402A0936502B09366029CE088E166
:1037B0000FB6F894A895809360000FBE90936000B8
:1037C000FFCF80913E0208950895CF93DF9321E0CB
:1037D0002093E9002FEF3091E800215035FD06C01D
:1037E00035ED3A95F1F700002111F5CF2091E80071
:1037F00025FF14C0EC0140E050E068E070E00E945A
:10380000AF1E8091E8008E778093E80088E0FE018B
:10381000A6E3B2E001900D928A95E1F7DF91CF9196
:103820000895809332027093340260933302809142
:103830005A02843001F582E08093E9008FEF909185
:10384000E800815095FD06C095ED9A95F1F70000CE
:103850008111F5CF8091E80085FF0DC040E050E078
:1038600063E070E082E392E00E94AF1E8091E80086
:103870008E778093E8000895BC0184E00C94111CBD
:10388000BC0183E00C94111C089581E897E00E942C
:10389000A00480915902811109C00E9440200E9419
:1038A0009D208091E20084608093E20008958DE77E
:1038B00097E00E94A00410925902089589E797E0CA
:1038C0000E94A0040C94EC1A85E797E00E94A004E3
:1038D0006091560281E0611101C080E00C94D71A1A
:1038E00081E797E00E94A00490915A0281E0943011
:1038F00009F080E0609156020C94DC1A20913102AC
:103900002F5F822F62E30E944C23992319F02093AA
:10391000310208951092310280913502882371F1AD
:1039200080915A02843041F58091E9008F70209196
:10393000EC00922F917020FD90E8892B93E09093FA
:10394000E9009091EB0090FF14C09091EE0097FF7A
:1039500010C09091E80095FF03C01092F100F9CFDC
:103960009091E80090FF05C09091E8009E779093B9
:10397000E8008F708093E90010923502089542E0CC
:1039800061EC81E00E94B91F42E261EC82E00E949A
:10399000B91F42E261EC83E00E94B91F90915A0284
:1039A00081E0943009F080E0609156020C94E51AB1
:1039B00080915C02833009F461C030F4813071F091
:1039C000823009F49AC008958A3009F486C08B3099
:1039D00009F46CC0893009F0A8C020C080915B0256
:1039E000813A09F0A2C08091E800877F8093E800C7
:1039F00080915F0290916002892B21F468E086E358
:103A000092E003C060E080E090E070E00E94FA1E67
:103A10008091E8008B778093E800089580915B02A5
:103A2000813209F082C080915F029091600202971A
:103A300008F07BC08091E800877F8093E800809148
:103A4000E80082FD05C080915A028111F8CF6DC057
:103A50002091F3008091F20090E0922B029731F4D4
:103A60008091F100813011F0863021F48091F100D5
:103A700080933E028091E8008B7753C080915B0277
:103A8000813A09F052C080915F0290916002892BC7
:103A900009F04BC08091E800877F8093E800809117
:103AA000E80080FFFCCF8091100136C080915B025E
:103AB0008132D9F580915F0290916002892BA9F53E
:103AC0008091E800877F8093E8000E94EE1F80913C
:103AD0005D02809310010C94130A80915B02813285
:103AE00021F58091E800877F8093E8000E94EE1F17
:103AF00080915E0280933F02089580915B02813A3B
:103B0000A1F48091E800877F8093E8008091E8002D
:103B100080FFFCCF80913F028093F1008091E8000C
:103B20008E778093E8000C94EE1F08959FB7F89469
:103B3000109235029FBF90915A02943009F057C0FD
:103B40009091E9009F703091EC00232F217030FD9F
:103B500020E8922B23E02093E9002091EB0020FF46
:103B600043C02091EE0027FF3FC020913002222366
:103B700021F02091E80025FF37C01092300226E0A6
:103B80003091E80035FD15C030915A02343061F5AE
:103B90003091EB0035FD28C0215021F481E0809365
:103BA000300222C0EFE9FFE03197F1F700C00000DA
:103BB000E7CF8093F1008091E80085FD0AC08091F5
:103BC000E80080FFFCCF8091E8008E778093E800CA
:103BD00006C08FB7F89421E0209335028FBF9F7005
:103BE0009093E90080E008959F709093E9008FEF33
:103BF000089584B7877F84BF0FB6F894A895809105
:103C00006000886180936000109260000FBE90E0B9
:103C100080E80FB6F89480936100909361000FBE26
:103C20000C94E71A0E9440200E949D20E2EEF0E0F2
:103C300080818460808378940C94312384E091E0C7
:103C40000C94011A80915A028530C9F48DE697E0F0
:103C50000E94A00480915A02853079F40E94381B9A
:103C6000809158028823B1F30E94F91A882391F3B6
:103C70000E94991E0E94130AEDCF0C94631B0895B5
:103C800008950C94431E292F332723303105C9F0A2
:103C900060F42130310581F02230310509F041C056
:103CA0008BE590E023EB37E040C021323105E1F0B5
:103CB0002232310531F135C082E190E02EE038E06A
:103CC00034C099278130910549F028F0029749F5D1
:103CD000E5E8F7E005C0EFEAF7E002C0E1E9F7E068
:103CE000849190E09F0121C063307105D0F4660F8C
:103CF000771FFB01E357FE4F2081318189E090E07F
:103D000014C06330710568F4FB01EE0FFF1FE95723
:103D1000FE4F20813181FB01EC57FE4F808190E006
:103D200004C080E090E020E030E0FA01318320839D
:103D3000089580E189BD82E189BD09B400FEFDCF0F
:103D40008091D8008F7D8093D8008091E0008260C0
:103D50008093E0008091E00081FDFCCF0895CF9238
:103D6000DF92EF92FF920F931F93CF93DF93EC01BB
:103D70008B017A010E940D20811133C0E114F104FE
:103D800039F0F70180819181081B190BC80FD91FE9
:103D9000C12CD12C0115110519F18091E80085FD88
:103DA00016C08091E8008E778093E800E114F1045A
:103DB00049F0F70180819181C80ED91ED182C0825D
:103DC00085E00FC00E940D20882321F30AC089914D
:103DD0008093F10001501109FFEFCF1ADF0ADACF0B
:103DE00080E0DF91CF911F910F91FF90EF90DF90D6
:103DF000CF90089520916102309162022617370713
:103E000048F06115710539F42091E8002E77209370
:103E1000E80001C0B901FC0120E06115710579F1EC
:103E200080915A028823F1F18530F1F18091E80008
:103E300083FD3CC08091E80082FD2EC08091E800A7
:103E400080FFEBCF2091F3008091F20090E0922B65
:103E50006115710551F08830910538F42191209356
:103E6000F100615071090196F3CF21E0089709F044
:103E700020E08091E8008E778093E800CECF21117A
:103E8000CFCF0AC080915A02882361F0853061F05B
:103E90008091E80083FD0AC08091E80082FFF2CFA4
:103EA00080E0089582E0089583E0089581E0089518
:103EB00020916102309162022617370748F06115A0
:103EC000710539F42091E8002E772093E80001C0B5
:103ED000B901FC0120E06115710591F180915A0250
:103EE000882309F440C0853009F43FC08091E80080
:103EF00083FD3DC08091E80082FD2FC08091E800E5
:103F000080FFE9CF2091F3008091F20090E0922BA6
:103F10006115710559F08830910540F42491209382
:103F2000F1003196615071090196F2CF21E00897B6
:103F300009F020E08091E8008E778093E800CBCFF5
:103F40002111CCCF0AC080915A02882361F08530BC
:103F500061F08091E80083FD0AC08091E80082FF53
:103F6000F2CF80E0089582E0089583E0089581E033
:103F70000895982F973068F59093E900981739F0D5
:103F80007091EC002091ED005091F00003C0242FBF
:103F9000762F50E021FD02C09F5FECCF3091EB0007
:103FA0003E7F3093EB003091ED003D7F3093ED008C
:103FB0003091EB0031603093EB007093EC00209374
:103FC000ED005093F0002091EE0027FDE5CF80E05A
:103FD00008958F708093E90081E0089580915B02DD
:103FE00087FF11C08091E80082FD05C080915A02D0
:103FF0008111F8CF11C08091E8008B770BC08091C0
:104000005A02882349F08091E80080FFF8CF809120
:10401000E8008E778093E80008952091E4003091C5
:10402000E50095E64091EC00842F817040FF23C0AD
:104030008091E80080FD1DC080915A02882399F08C
:10404000853099F08091EB0085FD11C04091E4002E
:104050005091E5002417350729F3915011F09A018A
:10406000E1CF84E0089582E0089583E0089581E03F
:10407000089580E008954091E80042FFDDCF089563
:104080000E94AE200E94B620E0EEF0E080818160C8
:104090008083E8EDF0E080818F77808319BCA7ED05
:1040A000B0E08C918E7F8C9380818F7E8083109284
:1040B000590208950F931F93CF93DF930E94AE2070
:1040C0000E94B620C8EDD0E088818F7788838881F0
:1040D0008068888388818F7D888319BC10925A02FA
:1040E00010925602109258021092570200EE10E001
:1040F000F80180818B7F808388818160888342E0A2
:1041000060E080E00E94B91FE1EEF0E080818E7FE8
:104110008083E2EEF0E0808181608083808188602E
:104120008083F80180818E7F80838881806188838D
:10413000DF91CF911F910F910895E8EDF0E080811C
:104140008F7E8083E7EDF0E080818160808384E072
:1041500082BF81E0809359020C945A20E8EDF0E090
:1041600080818E7F80831092E20008951092DA00A1
:104170001092E10008951F920F920FB60F92112432
:104180002F933F934F935F936F937F938F939F935F
:10419000AF93BF93EF93FF938091E10082FF0BC039
:1041A0008091E20082FF07C08091E1008B7F8093C5
:1041B000E1000E947E1C8091DA0080FF1FC0809188
:1041C000D80080FF1BC08091DA008E7F8093DA00D8
:1041D0008091D90080FF0DC080E189BD82E189BD59
:1041E00009B400FEFDCF81E080935A020E94451C75
:1041F00005C019BC10925A020E94571C8091E10020
:1042000080FF19C08091E20080FF15C08091E2001C
:104210008E7F8093E2008091E20080618093E200D3
:104220008091D80080628093D80019BC85E080938B
:104230005A020E94641C8091E10084FF30C080918A
:10424000E20084FF2CC080E189BD82E189BD09B410
:1042500000FEFDCF8091D8008F7D8093D8008091A3
:10426000E1008F7E8093E1008091E2008F7E809359
:10427000E2008091E20081608093E200809156022A
:10428000882311F084E007C08091E30087FD02C01D
:1042900081E001C083E080935A020E94701C8091EB
:1042A000E10083FF29C08091E20083FF25C0809157
:1042B000E100877F8093E10082E080935A021092B0
:1042C00056028091E1008E7F8093E1008091E200B0
:1042D0008E7F8093E2008091E20080618093E20013
:1042E00042E060E080E00E94B91F8091F0008860A9
:1042F0008093F0000E945E1CFF91EF91BF91AF91FF
:104300009F918F917F916F915F914F913F912F91ED
:104310000F900FBE0F901F9018951F920F920FB61F
:104320000F9211242F933F934F935F936F937F933B
:104330008F939F93AF93BF93CF93DF93EF93FF93AD
:10434000C091E900CF708091EC00D82FD17080FD32
:10435000D0E81092E9008091F000877F8093F00010
:1043600078940E94D1211092E9008091F000886039
:104370008093F000CD2BCF70C093E900FF91EF91B7
:10438000DF91CF91BF91AF919F918F917F916F916D
:104390005F914F913F912F910F900FBE0F901F9003
:1043A00018951F93CF93DF93CDB7DEB7AA970FB6BB
:1043B000F894DEBF0FBECDBFEBE5F2E08091F100D7
:1043C000819322E0E336F207C9F70E94D81C80915E
:1043D000E80083FF2EC180915B0290915C02492F1F
:1043E00050E04A30510508F024C1FA01EE59FF4F60
:1043F0000C945823803821F0823809F01AC108C083
:104400008091570290915802992389F082600FC0E1
:1044100080915F028F70873008F00BC18093E900B4
:104420008091EB0085FB882780F91092E90090913C
:10443000E800977F9093E8008093F1001092F100DC
:10444000D1C0282F2D7F09F0F4C0882319F08230C5
:1044500061F0EFC080915D02813009F0EAC09330D5
:1044600009F080E0809358022EC080915D02811196
:104470002AC080915F028F702FEF280F263008F03E
:10448000D8C08093E9002091EB0020FF1CC093303E
:1044900021F48091EB00806214C09091EB00906158
:1044A0009093EB0021E030E0A90102C0440F551FBA
:1044B0008A95E2F74093EA001092EA008091EB00BF
:1044C00088608093EB001092E9008091E800877F7C
:1044D0008093E8000E94EE1FACC08111AAC0109129
:1044E0005D021F778091E3008078812B8093E30049
:1044F0008091E800877F8093E8000E94EE1F809102
:10450000E80080FFFCCF8091E30080688093E300A7
:10451000111102C082E001C083E080935A0289C079
:104520008058823008F085C080915D0290915E02D3
:104530008C3D53E0950779F583E08A838AE289838D
:104540004FB7F894DE01139620E03EE051E2E32FEE
:10455000F0E050935700E49120FF03C0E295EF7024
:104560003F5FEF708E2F90E0EA3010F0C79601C0E9
:10457000C0968D939D932F5F243149F74FBF809153
:10458000E800877F8093E8006AE270E0CE01019640
:104590000E94FA1E16C060915F0270916002AE0127
:1045A0004F5F5F4F0E94411EBC01892B09F441C03F
:1045B0009091E800977F9093E80089819A810E940A
:1045C000581F8091E8008B778093E80032C08038D4
:1045D00081F58091E800877F8093E8008091560202
:1045E0008093F1008091E8008E7772CF811121C015
:1045F00080915D0290915E0299270297D4F4809198
:10460000E800877F8093E80080915D0280935602E6
:104610000E94EE1F80915602811106C08091E30036
:1046200087FD02C081E001C084E080935A020E94AD
:10463000BF1C8091E80083FF0AC08091E800877F5B
:104640008093E8008091EB0080628093EB00AA9653
:104650000FB6F894DEBF0FBECDBFDF91CF911F9193
:104660000895CF9380915A028823A1F0C091E90068
:10467000CF709091EC00892F817090FD80E8C82B5D
:104680001092E9008091E80083FD0E94D121CF7053
:10469000C093E900CF910895991B79E004C0991F58
:1046A000961708F0961B881F7A95C9F7809508958C
:1046B000EE0FFF1F0590F491E02D0994FB01DC0142
:1046C00004C08D910190801921F441505040C8F7E9
:1046D000881B990B0895F999FECF92BD81BDF89A78
:1046E000992780B50895A8E1B0E042E050E00C942D
:1046F0009F23262FF999FECF92BD81BDF89A01978D
:1047000000B4021639F01FBA20BD0FB6F894FA9A19
:10471000F99A0FBE08950396272F0E947A230E94CC
:104720007923252F0E947A23242F0C947A23019633
:10473000272F0E947A230C947923DC01CB01FC0102
:10474000F999FECF06C0F2BDE1BDF89A319600B4EA
:0E4750000D9241505040B8F70895F894FFCFF5
:10475E00C8000502E11BE51B441C401C3C1CE41B6D
:10476E0001E200E900EA00B500B600B700CD008313
:10477E0001CC008A01920194012102230224022518
:10478E0002260227022A02B300B4006F00700081D5
:10479E008283E200E900EA00B500B600B700CD0062
:1047AE008301CC008A01920194012102230224028A
:1047BE002502260227022A02B300B4006F00700001
:1047CE0081828330313233379091929395949666ED
:1047DE0035349736403222740842082008C507DE69
:0447EE0007F70700C2
:00000001FF
